:020000041000EA
:1000000070020020D5000010DD000010DF0000109D
:1000100000000000000000000000000000000000E0
:10002000000000000000000000000000E1000010DF
:100030000000000000000000E3000010E5000010D8
:10004000E7000010E7000010E7000010E7000010D4
:10005000E7000010E7000010E7000010E7000010C4
:10006000E7000010E7000010E7000010E7000010B4
:10007000610E0010CD0E0010E7000010E700001028
:10008000E7000010E7000010E7000010E700001094
:10009000E7000010B50C0010690D0010E70000101B
:1000A000E7000010E7000010000000000000000062
:1000B0000000000000000000000000000000000040
:1000C0000348854600F0BAFA00480047891300103B
:1000D000700200200448804704480047FEE7FEE71E
:1000E000FEE7FEE7FEE7FEE7A50C0010C1000010EA
:1000F00030B50B46014600202022012409E00D46C0
:10010000D5409D4205D31D469540491B2546954047
:1001100040191546521E002DF1DC30BD03460B433D
:100120009B0703D009E008C9121F08C0042AFAD2AD
:1001300003E00B780370401C491C521EF9D2704733
:10014000D2B201E00270401C491EFBD2704700226F
:10015000F6E710B513460A4604461946FFF7F0FFC6
:10016000204610BDF0B50C465C4085B0E40FE407B6
:1001700003944C000026640859009446490802463E
:100180000296224321D062460A431ED06200570DD8
:100190004A000E032303550D012402462C49240571
:1001A000781B1B0B360B40182343264361460090F7
:1001B0001C46501AB44103D30098401C009002E042
:1001C000921800985B41002803DA0020014605B030
:1001D000F0BD0020012109050746864611E064466E
:1001E0001D46141BB54106D36546521BB3417446E8
:1001F00007430C43A646CD074008490828439218F8
:100200005B4105460D43EAD11046184313D06046C2
:10021000194650407140084306D06046101AB34159
:1002200006D20122002306E000220123DB0702E0C0
:100230000122D2435310009874460105381C6141D5
:10024000029C039D0019694100F055F8BFE70000CA
:10025000FD0300000EB5C217C10F5040CA07401879
:100260000021054B0293019200910A460B4600F0D3
:100270004FF803B000BD0000330400000EB505497F
:100280000291002100910A460B46019100F040F8CE
:1002900003B000BD330400004A0009030123090B29
:1002A0001B051943094B10B5520D9A4201DA002083
:1002B00010BD064B34339A4203DC9A1A00F00AF858
:1002C00010BD03495118884010BD0000FF03000015
:1002D000CDFBFFFF10B5202A04DB0846203AD040B2
:1002E000002110BD0B46D340D0402024A21A9140DB
:1002F0000843194610BD10B5002B08DA0024401C35
:10030000614192185B411A4301D14008400010BD81
:10031000F0B51FB482B005460C0003D0084600F0CB
:10032000B3FE02E000F0B0FE20300246009021460D
:10033000284600F095F9049B059A04460F46184399
:100340001143084314D0184610431BD00098402195
:100350000A1A18460599FFF7BDFF05460E46009A92
:100360000599049800F07CF9084305D0012004E0C9
:100370002046394607B0F0BD0020C11705430E43A3
:100380002C43374300990E986305401A7905E40A17
:1003900000220C43FD0A0A3002D500200146E9E79D
:1003A0000105101969410C9C0D9D00196941FFF769
:1003B000A2FFDFE7F0B507460846584087B0C00FF8
:1003C000049048000E46590040084908BC1A88416C
:1003D00005D2384631461E4617460B46024658009F
:1003E000400810434CD0300D039040055900400D9B
:1003F000490D0590401A0290402872DA1803012135
:10040000000B09050843019004980092002805D0CC
:1004100001995242002088410092019002984021A7
:100420000A1A0199009800F01BF905460C466B4624
:1004300007CB00F025F9C0197141039A0E0D002376
:10044000D71756401A467A40164344D0049A002AD9
:100450002DD0029A012A039A15DC1205C01A914187
:1004600001263605001C7141D20F059ED20700936C
:10047000019202962A462346FFF74AFF07B0F0BDD5
:1004800038463146FAE71605224A0F46B218C01A16
:10049000B74101210905001C4F4100187F41114659
:1004A00018187941E20F10436D19644113E0E20717
:1004B0006D0815436408C2071443039A0126120508
:1004C000C01A91413605001C7141CE0740083043E7
:1004D0004908C01851412A462346FFF70CFFCDE7D3
:1004E000FFE7049801224000C117121A00238B4134
:1004F00004983146C417381AA141EEE730B40124FC
:10050000E407634030BC55E730B40124E4076140A0
:1005100030BC4FE70000E0FFF0B51FB488B00B9986
:100520000998002448400999C00F490049080991D9
:10053000C0070B990090490049080B910999089848
:10054000A64608431CD00B990A98084318D009986E
:1005500001244000420D4800410D09982405000384
:10056000000B204309900B980003000B20430B90D5
:1005700050181C494018002201901446104605E00E
:10058000002001460DB0F0BD032801DA034600E06B
:1005900003239C46C11A0AAE0AE05F0008ADED5B7A
:1005A0004F00F75B7D430027AA187C41491C5B1E66
:1005B0006145F2DD410004AB5A522104120C0A439A
:1005C000240C401C0828DFDB01980290009970463B
:1005D00001910090059B049A07990698FFF798FEF1
:1005E000D0E700000DFCFFFF70B54B005B08034334
:1005F0000BD04B005C0D002633466542B341D41747
:10060000AD1AA34102DB0020014670BD120530186F
:10061000514170BD10B5002904DB0124E4074042BC
:100620008C412146002B04DB1C460123DB07524290
:10063000A341994200D1904210BD0000064C012513
:10064000064E05E0E36807CC2B430C3C984710347A
:10065000B442F7D3FFF738FDB8200010D8200010BF
:1006600010B5202A04DB0146203A9140002010BD3D
:10067000914020239C1A0346E3401943904010BD4B
:1006800010B5202A06DBCB170846203A1041C117C7
:100690000B4306E00B461341D0402024A21A9140A0
:1006A0000843194610BDFEB500231A461B1A8A419D
:1006B00003DB0020014603B0F0BD4A000D03012119
:1006C0002D0B0905520D0D43D10702D100186D41C4
:1006D000521E5110FF31FF310131002704463E46C2
:1006E0003846009701910246012100200905FFF7D5
:1006F000F1FDC3197141F818324684468E464A41CD
:1007000061462846611A904104D36046241A9541F7
:1007100076461F46241900986D41401C00903428ED
:10072000E1DDF91930467041091BA84103D20022CE
:10073000D243134601E00022134601980105381CFC
:100740007141FFF7D8FDB6E710B5134600224160AE
:100750008160002B01D0082422430124224302603F
:1007600010BD000010B5034800F008F80249086009
:1007700010BD0000200000201C000020F0B587B054
:100780000446002754480068217809040843524968
:100790000860207800281AD108464068617809016D
:1007A00008434D4948606178881CFFF753FD0246B5
:1007B0000B460591049000200121890700F05EFEA0
:1007C0000546FFF769FDC7B244494F4328E020784A
:1007D000012803D1A77841494F4321E0207802281E
:1007E00001D187031CE02078032801D1A78817E0F6
:1007F00039484068617809010843374948606178A1
:10080000881CFFF727FD02460B4605910490002047
:100810000121890700F032FE0546FFF73DFDC7B212
:100820002D480068A17908432B49086000BF2A4879
:1008300000684007C00F0028F9D127480068217AD6
:10084000090208432449086008460068E179090361
:10085000084321490860207A00281BDD217AC81E40
:10086000FFF7F8FC05462A460B46002001218907C0
:1008700000F004FE039102903846FFF7FFFC01915F
:100880000090039B029AFFF76DFC05910490FFF71F
:1008900003FD0746E07900281BDDE179C81EFFF75C
:1008A000D9FC05462A460B4600200121890700F0A5
:1008B000E5FD039102903846FFF7E0FC01910090BE
:1008C000039B029AFFF74EFC05910490FFF7E4FCAE
:1008D0000746384607B0F0BD0000024040420F0016
:1008E00010B50446002C04D00A2221460148FFF727
:1008F00015FC10BD6400002010B5154800780028D4
:1009000024D014480068401C12490860084600685A
:1009100005210902884205D20F4881880F4801F05D
:1009200029FB13E00B4800680521090488420DD318
:1009300008480068C911884205D2074881880748DD
:1009400001F018FB02E000200249086010BD000021
:1009500050000020540000206400002000C000402F
:1009600010B501F0EFFA02A000F07EFB10BD000010
:10097000E794B5E588BAE6BF80E5B7B2E590AFE5A4
:100980008AA85C6E0000000010B5002005490870C0
:1009900005490860054801F0E1FA05A000F064FB94
:1009A00010BD0000500000205400002000C0004096
:1009B000E794B5E588BAE6BF80E5B7B2E5819CE685
:1009C000ADA25C6E0000000010B502460F2A14DDD7
:1009D0001348806B1346103B5C000323A3409843ED
:1009E0000F4B98631846806B1346103B5C000B4618
:1009F000A34018430A4B98630FE00948406B54002A
:100A00000323A3409843064B58631846406B540099
:100A10000B46A3401843024B5863002010BD000052
:100A20000010024001460448406801228A401040FC
:100A3000C840C0B27047000000100240FFB5044635
:100A40000D461E460B9F00212046FFF7BDFF012DDE
:100A500010D1012F0ED14F4800690121A1408843D8
:100A60004C490861084640690121A14008434949B1
:100A700048613BE0012D10D1002F0ED1454800699F
:100A80000121A1408843434908610846406901218A
:100A9000A14088433F49486128E0002D14D1012F2F
:100AA00012D13C4840690121A1408843394948613D
:100AB000084600690121A1400843364908610998A8
:100AC00048620298086311E0002D0FD1002F0DD16C
:100AD000304800690121A14088432E490861084639
:100AE00040690121A14088432A494861022E0ED164
:100AF000284880690121A140884326498861084629
:100B0000C1690120A04081432248C1611FE0002E3D
:100B10000ED1204880690121A14008431D49886108
:100B20000846C0690121A14088431A49C8610EE006
:100B3000012E0CD1174881690120A040814315483E
:100B40008161C0690121A14008431249C86111486F
:100B5000816A0120A04081430E488162806A0A991F
:100B6000C907C90FA14008430A4988620846C06AFC
:100B70000121A14088430749C8620846C06A0A9912
:100B80008907C90FA14008430249C862002004B088
:100B9000F0BD000000100240012907D1074A526849
:100BA000012383401A43054B5A6006E0034A52680A
:100BB000012383409A43014B5A6070470010024062
:100BC00000B503461846FFF72DFF012803D118464C
:100BD00000F00AF807E01846FFF724FF002802D1CA
:100BE000184600F00BF800BD034949680122824015
:100BF0009143014A5160704700100240034949681F
:100C0000012282401143014A5160704700100240A6
:100C100000207047C206D20E01219140014A1160A6
:100C20007047000080E200E0C206D20E0121914030
:100C3000014A11607047000080E200E0C206D20E57
:100C400001219140014A11607047000080E100E0FD
:100C5000C206D20E01219140014A11607047000086
:100C600080E100E0C206D20E01219140014A1160EC
:100C70007047000000E100E0C206D20E0121914061
:100C8000014A11607047000000E100E0014604489D
:100C9000406901228A401043014A50610020704798
:100CA00000000240014802490860704700E1F50574
:100CB0005C00002000B501200449C86004480068B9
:100CC000401C0349086000F06FF800BD0080004040
:100CD0004400002070B504460820FFF7D7FF152018
:100CE000FFF7B6FF1520FFF79FFF7D21C9000B48D6
:100CF0000068FFF7FDF960430546294608A000F0AB
:100D0000B3F9012229460C48FFF71EFD1520FFF715
:100D1000B3FF214609A000F0A7F970BD1C00002018
:100D200054494D455230E9878DE8A385E8BDBDE5BE
:100D300080BC3A2025640A000080004054494D459B
:100D400052305F496E6974E5AE8CE68890EFBC8CDA
:100D5000E4B8ADE696ADE591A8E69C9F3A202564FF
:100D6000206D730A0000000001200449C860044897
:100D70000068401C02490860704700000090004075
:100D80004C000020004870473400002010B50621B8
:100D90000348FFF7DCF908210248FFF7D8F910BD36
:100DA000340000203A0000202B480078401C2A49DB
:100DB000087008464078401C487008468078401CFF
:100DC00088700846C078401CC87008460079401CEE
:100DD00008710846C088401CC88008460078022870
:100DE00004DB0020087001201C4908701A48407874
:100DF000062805DB00201849487001201749487073
:100E0000154880780A2805DB0020134988700120E6
:100E1000124988701048C078142805DB00200E495C
:100E2000C87001200D49C8700B480079642805DBA3
:100E30000020094908710120084908710648C08846
:100E40007D21C900884205DB00200349C8800120BC
:100E500002494871704700003A0000203400002029
:100E600010B500240C20FFF7D5FE0120800700F00C
:100E700062F8032806D101208007406804218843D6
:100E8000090748600120800700F055F8022805D0C6
:100E90000120800700F04FF8062816D101208007B6
:100EA0004068400840000121890748600846006802
:100EB000C4B221460120800700F0C4F80120800759
:100EC0004068012108438907486010BD10B500241F
:100ED0000D20FFF79FFE144800F02DF8032805D1E0
:100EE00011484068042188430F4948600E4800F0CB
:100EF00022F8022804D00C4800F01DF8062812D170
:100F000009484068400840000749486008460068B2
:100F1000C4B22146044800F095F803484068012116
:100F200008430149486010BD00100040014648696F
:100F30008006C00F7047014688680007400F704761
:100F400070B504460D461348844206D10D20FFF7C4
:100F500075FE0D20FFF75EFE09E001208007844248
:100F600005D10C20FFF76AFE0C20FFF753FE6068E6
:100F70002978084360600748844203D10D20FFF7B9
:100F800071FE06E001208007844202D10C20FFF7A9
:100F900069FE70BD00100040F8B504460D46012002
:100FA000800784420BD10020FFF770FE0121022050
:100FB000FFF70AFD01210320FFF706FD0DE01F48A2
:100FC00084420AD10120FFF761FE01210C20FFF7C6
:100FD000FBFC01210D20FFF7F7FC606BC007C00F81
:100FE000002801D1102700E00D2715486968006826
:100FF000FFF77EF839460090FFF77AF8401E86B278
:101000001120304020621120000230400012606246
:10101000A068E968097889010843A060E8688078D9
:10102000012803D1A06801210843A060287A012883
:1010300003D12069202108432061F8BD0010004041
:101040001C00002000B503460A4600BF1846FFF703
:101050006DFF0028FAD01146184600F002F810463D
:1010600000BD0160704700000FB410B503A9044B28
:10107000044A029800F0CCF810BC08BC04B0184731
:10108000751300102C0000202021020C01D010212B
:101090001046020A01D010460839020901D0104654
:1010A000091F820801D01046891E420801D0881EFF
:1010B0007047081A704700004900CA020243100036
:1010C00000D004204A0D01D001221043044A490DEA
:1010D000914201D102210843012800D10520704727
:1010E000FF070000F8B504464F1EC8000838211855
:1010F00015461E46086849683A4606239A4310D0AA
:101100002A463346FFF708FA3A46D200083AA318AF
:101110001A687F1E5B68FFF74DF906223B46934332
:10112000EED1022F23D0042F11D0062F2FD12A4623
:101130003346FFF7F1F9E36AA26AFFF73BF92A4663
:101140003346FFF7E9F9636A226AFFF733F92A4663
:101150003346FFF7E1F9E369A269FFF72BF92A4665
:101160003346FFF7D9F963692269FFF723F92A4665
:101170003346FFF7D1F9E368A268FFF71BF92A4667
:101180003346FFF7C9F963682268FFF713F9F8BD22
:10119000002210B5134610460149FEF7E3FF10BDCB
:1011A0000000F03F10B5FFF705F910BD002210B5A3
:1011B000134610461146FEF7D5FF10BD10B50721A6
:1011C000024A00200907FFF70FFA10BD01030000D3
:1011D000034A10B500201107FFF706FA10BD000002
:1011E00001FDFFFF02E008C8121F08C1002AFAD162
:1011F00070477047002001E001C1121F002AFBD197
:10120000704700000149086070470000600000203E
:10121000FFB58DB00446002506E025280AD0109AB7
:101220000F999047641C6D1C20780028F5D1284642
:1012300011B0F0BD00270121484A009700E00743A4
:10124000641C23780846203B98401042F7D1207850
:101250002E2817D1042007436078641C2A280CD15B
:101260000E98641C02C800910E900BE000990A22AF
:10127000514330394018641C0090207801463039C1
:101280000929F3D920780028D1D0642808D069280A
:1012900006D075281ED0109A0F9990476D1C5BE000
:1012A0000A200E99019001C90E91002802DA4042ED
:1012B0002D2102E0390504D52B216A461172012146
:1012C00003E0F90704D02021F7E70BAE0B910DE006
:1012D0000021FAE70A200E99019001C90E91F7E763
:1012E0000199FEF705FF3031761E31700028F7D1E5
:1012F00003A8801B20300190780701D5009801E0F9
:10130000012000900199884201DD401A00E0002090
:101310000027009006E002A8109AC05D0F99904740
:101320006D1C7F1C0B988742F5DB04E0109A30207F
:101330000F9990476D1C0099481E00900029F5DC1C
:1013400005E03078109A761C0F9990476D1C019932
:10135000481E01900029F4DC641C65E7092801009F
:101360000248034948611020086170471372070062
:1013700000E0004070B504460D46E1B20148FFF7B9
:1013800061FE70BD0010004086B0FFF741FCFFF722
:10139000E9F901200021009102230A4601910290FF
:1013A0001320FFF74BFB00211320FFF7F5FB2D491E
:1013B0002D48FFF7F1FD2D492B48FFF7C1FD012016
:1013C000FFF788FCFFF7E2FC00F08AFD284A07CA15
:1013D00003AB07C303A8FFF783FAFFF7C1FA40E0A6
:1013E000FFF7D0FC04462078002801D000202070B0
:1013F000A078002801D00020A0702079002801D01A
:1014000000202071607900282AD01A480078401CFA
:1014100018490870084600780A280BDC164800783E
:10142000002804D1012014490870FFF799FAFFF74A
:1014300063FA10E00F480078142809DC0E480078A1
:10144000012808D100200C490870FFF79DFA02E03E
:101450000020084908701320FFF7B2FB00206071DC
:1014600000BFBDE708000020001000401800002069
:101470001C2000100000002001000020F0B51FB467
:1014800096B084460C460246199D18980390490070
:1014900068006300490840080193002A01D0012632
:1014A00000E000269E19FE4BF6185B109E422BD3DF
:1014B0006E00039F0296002F00D00127F719F84E07
:1014C000F84BBE199E421FD3039E0346F64F33438B
:1014D00009D03B469C4201D1002A04D0019B002A3E
:1014E00005D0012604E0002039461BB0F0BD0026DF
:1014F0009E19EE4B9E4207D8039F029E002F00D0FC
:101500000127F6199E4207D92B4660462146189AB4
:10151000FFF748FE1BB0F0BD0023002C29DAE44E93
:10152000B04226DAE34EB04201DB022321E0DE4E78
:10153000B0421EDBE04E070DBE19142E09DD342724
:10154000BF1B039EFE400196BE40039FBE420BD0D0
:101550000FE0039F002F0CD11427BF1B0646FE404F
:101560000196BE40864204D1019BDE07F60F02239E
:101570009B1B0E46164318D1002D16DA002C03D003
:10158000022B01D0012B06D00220FFF73BFEFFF714
:10159000FFFD1BB0F0BD0220FFF734FEFFF7F8FDA2
:1015A0000122D20751401BB0F0BD039E002E61D135
:1015B000BF4EB04220D1C148844201D1002A08D098
:1015C000B948814209DB002D10DB189829461BB071
:1015D000F0BD0020B4491BB0F0BD002D06DA012299
:1015E0002946D207189851401BB0F0BDB449794440
:1015F000086849681BB0F0BDAB4FB84225D1002D3B
:101600001FDA002904D0B14212D1002A09D018E013
:10161000002A72D1A649E20F0020D20711431BB065
:10162000F0BD0020E20F0146D20711431BB0F0BD10
:10163000B14206DA234600203946FEF793FD1BB07F
:10164000F0BD104621461BB0F0BDB14212DA0126B2
:10165000B607B54203D1234610461946FEE3994E1C
:10166000B54207D1261E05DB1046314600F014FCBA
:101670001BB0F0BD67007F081646002A40D1002944
:101680000AD08B4A914229D1002C0EDD002D1CDBA3
:10169000002011461BB0F0BD022B16D0002C14D038
:1016A000012B12D1002C14DB0FE0002C28DA002DC6
:1016B00009DB012B03D000207D491BB0F0BD0020C9
:1016C00081491BB0F0BD012B03D0002001461BB0A7
:1016D000F0BD00200121C9071BB0F0BD724A914244
:1016E0000ED1002C01DA002B17D0022B06D00020DF
:1016F000C043FEF7AFFD1BB0F0BD90E20120F8E75C
:10170000E217521C94461A4307D000220892664CF6
:1017100062465B1E1A4307D009E00120FFF772FD05
:10172000FFF744FD1BB0F0BD0022644C0892674AED
:1017300090427DDD664B674A98421FDD914202DC94
:10174000002D05DB4DE05848814217DB002D48DDB8
:101750000220FFF757FDFFF731FD05460E46002238
:10176000534B21460898FEF7D7FE084671004908FA
:10177000C00FC007014328461BB0F0BD914215DAE7
:10178000002D2EDA0220FFF73DFDFFF717FD05467D
:101790000E460022464B21460898FEF7BDFE720019
:1017A0005208C80FC0070243114617E03E4B99424A
:1017B00023DD002D15DD0220FFF724FDFFF7FEFCE1
:1017C00005460E4600223A4B21460898FEF7A4FE35
:1017D000084671004908C00FC007014328461BB0E6
:1017E000F0BD0220FFF70EFDFFF7F2FC49004908AB
:1017F000E20FD20711431BB0F0BD0022304639463C
:10180000FEF77CFE012205460E46D243FEF7ECFEB3
:10181000314A324BFEF778FE2A463346FEF77CFE0D
:101820000022284BFEF770FE07462A46334600E0AA
:1018300064E0039110461946FEF76EFE3A46039B9C
:10184000FEF76AFE0746032209915207244B2846F9
:101850003146FEF761FE07910C90224A204B384634
:101860000999FEF759FE074601911F4A1F4B28466A
:101870003146FEF751FE3A46019BFEF73FFE074612
:101880000B460246099107990C98FEF793FD002537
:101890000E462846079B0C9AFEF730FE3A4627E094
:1018A000FFFF1F00FFFF0F000000F03F0000E0FF00
:1018B0000000F07F0000404301FCFFFF0000F0BF8C
:1018C000BE0A00000000E03F0000F0FF0000E04121
:1018D0000000F043FFFFEF3F555555555555D53F97
:1018E0004715F73FFE822B6544DF5DF80BAE543E93
:1018F000099BFEF709FE02460B4652E10125002036
:101900002D05A94207DA352230463946FEF76CFE2E
:1019100006463420C0430A151218FE4810180390DA
:101920000803FD49000B01430F46FC49884201DCD6
:10193000002003E0FA49884202DA0120119005E014
:10194000002011900398401C7F1B0390119805976D
:10195000C200F4480F927844801843680268394600
:1019600030460D930292FEF7C9FD07910C90304668
:101970000D9B029A0599FEF71DFD02460B460020BD
:10198000E549FEF7EFFB09910490079B0C9AFEF7DF
:10199000C3FD129000201090E3480D467844006883
:1019A0000E90012178104907084311990D9B890475
:1019B00040180121C90447183946029A0E98FEF7CB
:1019C0009DFD3246059BFEF79FFD02460B462946CC
:1019D0001098FEF7A1FD064602913B4629460E9A55
:1019E0001098FEF799FD079B0C9AFEF78DFD324685
:1019F000029BFEF783FD099B049AFEF78DFD05917E
:101A0000129A0A902B4610461946FEF785FD0646A7
:101A10000246C6480F460B4606217844FFF762FB94
:101A200032463B460091049010461946FEF774FD7D
:101A3000009B049AFEF770FD06460F462B4619469A
:101A4000129A1098FEF7B6FC059B0A9AFEF764FD01
:101A500032463B46FEF7AEFC109A079104902B46A7
:101A600010461946FEF758FDB14E00223346099143
:101A70000290FEF79FFC079B049AFEF79BFC002058
:101A80000746024633460091FEF738FD099B029A4D
:101A9000FEF734FD079B049AFEF736FD06460D91CE
:101AA0003A462946009B1098FEF736FD07910C90A8
:101AB0002B463046129A0D99FEF72EFD05460E462E
:101AC0003A46009B05990A98FEF726FD33462A46BA
:101AD000FEF770FC02460B460746099107990C98E1
:101AE000FEF768FC00250E462846079B0C9AFEF779
:101AF00005FD3A46099BFEF707FD074607220991B7
:101B000052078C4B31462846FEF706FD07910090A0
:101B1000894A884B38460999FEF7FEFC0746019131
:101B2000864A874B31462846FEF7F6FC3A46019B2B
:101B3000FEF740FC834B7B440F9A9B181A685B6846
:101B4000FEF738FC029009910398FEF783FB05919C
:101B50000490099B029A07990098FEF72BFC7A4B98
:101B60007B440F9A9B181A685B6817460393FEF72D
:101B700021FC059B049AFEF71DFC0E462846059B9A
:101B8000049AFEF7BBFC3A46039BFEF7B7FC079BA3
:101B9000009AFEF7B3FC099B029AFEF7B5FC0246D9
:101BA0000B46199900200C900F461898FEF7B4FCCC
:101BB000029104903B460C9A19991898FEF79EFCE6
:101BC0002A463346FEF7A8FC029B049AFEF7F2FB76
:101BD00009910E902A46334639460C98FEF79CFC34
:101BE00006460F46099B0E9AFEF7E4FB574A0D4640
:101BF000914220DB5242AA18024310D132463B46A2
:101C0000FEF77CFC04900391514A524B09990E98BF
:101C1000FEF7D0FB039B049AFEF7FCFC1ED20220C9
:101C2000FFF7F0FAFFF7CAFA49004908E20FD207B6
:101C300011431BB0F0BD6A00474B52089A420DD3C6
:101C4000464AAA18024300D0CBE532463B46FEF78F
:101C500055FC099B0E9AFEF7DDFCF5D968000023C0
:101C600040082C490393020D3D4B5218984223DD46
:101C700001200005521CD04042195000400D401870
:101C800038497944096813468C463749C1408B432B
:101C900012030121120B090551181422101AC14018
:101CA0000391002D01DA48420390624630463946DE
:101CB000FEF724FC06460F4632463B4609990E982D
:101CC000FEF778FB00252A46284B28460591FEF7AB
:101CD00023FC07910C90264A264B28460599FEF7CF
:101CE0001BFC0091029032463B4628460599FEF7C0
:101CF00005FC099B0E9AFEF707FC1F4A1F4BFEF7D7
:101D00000BFC009B029AFEF755FB07460B4602466A
:101D1000099135E001FCFFFF0000F03F8E980300C1
:101D20007AB60B00CE060000100700003A0600004D
:101D30000000084009C7EE3FFD033ADCF5015B14E3
:101D4000E02F3EBE0E050000D404000000009040CD
:101D5000FE822B654715973C00CC904000346F3FC6
:101D60000000E03F2A040000FFFF0F00432EE63F83
:101D7000396CA80C615C20BEEF39FAFE422EE63FBA
:101D800007990C98FEF716FB05460E46079B0C9A22
:101D9000FEF7B4FB3A46099BFEF7B6FB09912A46CB
:101DA00033460E9010461946FEF7B6FB074602462C
:101DB0002F480B46059105217844FFF793F93A46E1
:101DC000059BFEF7A9FB2A463346FEF79DFB074617
:101DD000019128463146099B0E9AFEF79DFB099B0F
:101DE0000E9AFEF7E7FA012304910C9000229B075C
:101DF00038460199FEF782FB05910E903A46284637
:101E00003146019BFEF788FB059B0E9AFEF7AAF967
:101E1000049B0C9AFEF772FB2A463346FEF76EFBD4
:101E20000022144BFEF770FB064603980D46000592
:101E300041190915002912DC30462946039AFEF79C
:101E4000D3FBFFF739F9042801D1FFF7C1F9304678
:101E50002946039AFEF7C8FB064601E004E029186C
:101E60000B46324621460898FEF756FB1BB0F0BDE4
:101E7000CC0200000000F03F10B5044601E0FFF77F
:101E800079FA2078641C03490028F8D10A20FFF76A
:101E900071FA10BD2C000020F8B506460C46FEF77E
:101EA00002FC051E0F4600D00120014349000B48EB
:101EB0004908411AC90F0DD0002E01D0012100E0C0
:101EC00000210C4361004908401AC00F02D10120D3
:101ED000FFF798F928463946F8BD00000000F07F6A
:101EE00010B50220064908600648406906490843C3
:101EF00004494861FFF734FA04A0FFF7BDFF10BDA5
:101F0000003002400000024003500000454E5331B3
:101F1000202D20574156455F47454E455241544F6D
:101F2000525F4452495645525F415F546573742075
:101F30002D20245265766973696F6E3A20523030D5
:101F4000310A00000120034908700020024908609E
:101F50007047000050000020540000200021C163A1
:101F600000BF03E0C16100220262491C4029F9DB85
:101F700070470000F8B504460D460026002716A05D
:101F8000FFF77AFF6420A0602020A061A061642098
:101F900020616061502020600420E063002002E0A6
:101FA000E0612562401C4028FADB1920C001606214
:101FB0000020A062E0620120206300206063A06333
:101FC00001206060002F04D00BA0FFF755FF012611
:101FD00000273046F8BD00000AE9A9B1E58AA8E566
:101FE00099A841E6ADA3E5BCA6E6B3A2E6B58BE8A9
:101FF000AF955C6E000000000AE99499E8AFAF204D
:102000003A20E9A9B1E58AA8E599A841E6B58BE8A7
:10201000AF95E5A4B1E8B4A50A0000006400E803A8
:102020008000640032000000000000000000F03F6B
:10203000000000000000F83F000000000000000069
:102040000000004003B8E23F000000000000000074
:1020500006D0CF43EBFD4C3E033333333333E33F02
:10206000FFAB6FDBB66DDB3F4D268F515555D53F2E
:1020700001411DA96074D13F65DBC9934A86CD3FFC
:10208000EF4E454A287ECA3F3E5555555555C53FEA
:1020900093BDBE166CC166BF2CDE25AF6A56113FDC
:1020A000F16BD2C541BDBBBED0A4BE726937663EDE
:1020B0000000000000000000D820001000000020F8
:1020C00064000000E41100103C21001064000020B6
:1020D0000C020000F41100100000000002000100DA
:1020E0000000000000C20100000000000400002009
:1020F00005000000000000000003000000000000D8
:1021000000000000000000000000000000000000CF
:1021100000000000000000000000000000000000BF
:1021200000000000000000000000000000000000AF
:0C21300000E1F50500E1F50500000000ED
:04000005100000C126
:00000001FF
